:020000040000fa
:080000000414040000000000dc
:020000040000fa
:1004000000000000000000000000000000000000ec
:1004100000000000000000000000000000000000dc
:1004200000000000000000000000000000000000cc
:1004300000000000000000000000000000000000bc
:10280000ffffff00ffffff008fdf2000807f24001d
:1028100000018800000000000a0007001100070006
:10282000000020000000e000020032000000020072
:1028300000000000e05c0200000000000040da0040
:102840000000fe004440a900c03a20000000e00063
:102850000300320000002000a00188004440a800ce
:1028600000000600a0f0260001002000160037003e
:1028700062004000e0804800910188009001ba00a9
:1028800062004000e0804800910188009002ba0098
:1028900062004000e08048000002eb006028e10098
:1028a00005003a008301e9000700330003800900b6
:1028b0000059eb00040037006128e10001003200fc
:1028c0000082eb0005000700910188001001ba00aa
:1028d0000200e000e6ff3a000000050091018800d8
:1028e0008002780062004000e08048003559ba005c
:1028f0008301e900080032002559ba008301e9008c
:10290000050032000400e000f4ff320015d9ba00df
:102910008301e900f1ff3a00000006001667040099
:10292000000000003c67040000000000ce480400e6
:10293000000000002648040000000000889fbe0040
:10294000e30440000900a100808f54004a003600d3
:10295000e38f540001003e004900200082498000be
:102960000200e00002003200820078000c00370014
:102970002193200003003700908f5400230036007d
:102980008080e800110078000000e000faff3a00c3
:102990000f003700908f54001c0036008080e80044
:1029a000110078000000e000faff3a001201780000
:1029b0002193200003003700908f5400130036004d
:1029c0008080e80011007800820f5000faff3a0082
:1029d00078498000890f5400010031000904780013
:1029e000080078005b0007000000e00004003a00e7
:1029f000890f5400200032000804d100f5ff370091
:102a0000081878001f000700d4ff37001101780074
:102a10009201780064805100890f5000030031005a
:102a2000120090008008780007003700090041007c
:102a3000800878009201900013009800110078003f
:102a40001288140009097800910078000100e00064
:102a500005003200110090000000e000020032008a
:102a60000180e800010037000000eb008049880089
:102a70000280e800010037000000eb004f04be00b8
:102a8000000006000000e000310032008080e90014
:102a900091027800e38f52002d0036000508a30054
:102aa0002b003a00924980000200e0000200320050
:102ab000828f50000400310002087800914988009c
:102ac0001600370003017800920190000300e00037
:102ad00002003200818f5100faff390012027800a3
:102ae00004004100808f500019003900810f500010
:102af00003003a0005094200820078000700370011
:102b00000300e0000300320005804000808f510088
:102b10000f003900930098001101980011019000f6
:102b20000200e0000a00320011804000820f5000d5
:102b300007003a00009320000008eb00110090000d
:102b4000110178009008410010009000900098005a
:102b5000000006000000e00003003400040007004d
:102b6000e10f400001003a000000eb000000060009
:102b7000889fbe00800478002c09e20004003a001f
:102b80000000eb00100007000000e0000a00350024
:102b9000604980000900e00002003a00000478006b
:102ba0000600370000047800090040000600070016
:102bb0000000e00001003d000084eb000800780008
:102bc0004f04be0000000600800078000000e00016
:102bd00004003a0000a1200060498800010178004b
:102be000060037000081eb0080df2000808f50005e
:102bf00002003e00614988000001eb0002007800fd
:042c000000000600ca
:020000040000fa
:020000040005f5
:0457f800fe9300001c
:020000040000fa
:020000040005f5
:0457fc007f3e0000ec
:020000040000fa
:10000800d66f0000d66f0000d66f0000d66f0000d4
:10001800d66f0000d66f0000d66f0000d66f0000c4
:10002800d66f0000d66f0000d66f0000d66f0000b4
:10003800d66f0000d66f0000d66f0000d66f0000a4
:10004800f0660000d66f0000d66f0000d66f000083
:10005800d66f0000d66f0000d66f0000d66f000084
:10006800d66f0000d66f0000d66f0000d66f000074
:10007800d66f0000d66f0000d66f0000d66f000064
:10008800d66f0000d66f0000d66f0000d66f000054
:10009800d66f0000d66f0000d66f0000d66f000044
:1000a800d66f0000d66f0000d66f0000d66f000034
:1000b800d66f0000d66f0000d66f0000d66f000024
:1000c800d66f0000d66f0000d66f0000d66f000014
:1000d800d66f0000d66f0000d66f0000d66f000004
:1000e800d66f0000d66f0000d66f0000d66f0000f4
:1000f800d66f0000d66f0000d66f0000d66f0000e4
:10010800d66f0000d66f0000d66f0000d66f0000d3
:10011800d66f0000d66f0000d66f0000d66f0000c3
:10012800d66f0000d66f0000d66f0000d66f0000b3
:10013800d66f0000d66f0000d66f0000d66f0000a3
:10014800d66f0000d66f0000d66f0000d66f000093
:10015800d66f0000d66f0000d66f0000d66f000083
:10016800d66f0000d66f0000d66f0000d66f000073
:10017800d66f0000d66f0000a4360000d66f0000ce
:10018800d66f0000d66f0000d66f0000d66f000053
:10019800d66f0000d66f0000d66f0000d66f000043
:1001a800d66f0000d66f0000d66f0000d66f000033
:1001b800d66f0000d66f0000d66f0000d66f000023
:1001c800d66f0000d66f0000d66f0000d66f000013
:1001d800d66f0000d66f0000d66f0000d66f000003
:1001e800d66f0000d66f0000d66f0000d66f0000f3
:0801f800d66f0000d66f000075
:020000040000fa
:10020800d66f0000d66f0000d66f0000d66f0000d2
:10021800d66f0000d66f0000d66f0000d66f0000c2
:10022800d66f0000d66f0000d66f0000d66f0000b2
:10023800d66f0000d66f0000d66f0000d66f0000a2
:10024800f0660000d66f0000d66f0000d66f000081
:10025800d66f0000d66f0000d66f0000d66f000082
:10026800d66f0000d66f0000d66f0000d66f000072
:10027800d66f0000d66f0000d66f0000d66f000062
:10028800d66f0000d66f0000d66f0000d66f000052
:10029800d66f0000d66f0000d66f0000d66f000042
:1002a800d66f0000d66f0000d66f0000d66f000032
:1002b800d66f0000d66f0000d66f0000d66f000022
:1002c800d66f0000d66f0000d66f0000d66f000012
:1002d800d66f0000d66f0000d66f0000d66f000002
:1002e800d66f0000d66f0000d66f0000d66f0000f2
:1002f800d66f0000d66f0000d66f0000d66f0000e2
:10030800d66f0000d66f0000d66f0000d66f0000d1
:10031800d66f0000d66f0000d66f0000d66f0000c1
:10032800d66f0000d66f0000d66f0000d66f0000b1
:10033800d66f0000d66f0000d66f0000d66f0000a1
:10034800d66f0000d66f0000d66f0000d66f000091
:10035800d66f0000d66f0000d66f0000d66f000081
:10036800d66f0000d66f0000d66f0000d66f000071
:10037800d66f0000d66f0000a4360000d66f0000cc
:10038800d66f0000d66f0000d66f0000d66f000051
:10039800d66f0000d66f0000d66f0000d66f000041
:1003a800d66f0000d66f0000d66f0000d66f000031
:1003b800d66f0000d66f0000d66f0000d66f000021
:1003c800d66f0000d66f0000d66f0000d66f000011
:1003d800d66f0000d66f0000d66f0000d66f000001
:1003e800d66f0000d66f0000d66f0000d66f0000f1
:0803f800d66f0000d66f000073
:020000040000fa
:102c04000d0a00002a2a00002a2a00002a200000b7
:102c1400555300004220000045720000726f00000e
:102c2400722000002d200000646500007669000019
:102c34006365000020720000657100007569000082
:102c44007265000073200000746f00006f200000a4
:102c54006d75000063680000206300007572000059
:102c6400726500006e740000202a00002a2a000009
:102c74002a2a00000d0a0000000d00000a2a0000a4
:102c84002a2a00002a2a000020550000534200008e
:102c940020450000727200006f720000202d0000b9
:102ca400206800007562000073200000617200005b
:102cb400652000006e6f0000742000007375000032
:102cc400707000006f7200007465000064200000e2
:102cd4002a2a00002a2a00002a0d00000a00000007
:102ce4000d0a00002a2a00002a2a00002a200000d7
:102cf400555300004220000045720000726f00002e
:102d0400722000002d200000646500007669000038
:102d14006365000020690000732000006e6f0000ee
:102d24007420000073750000707000006f72000062
:102d340074650000642000002a2a00002a2a00008a
:102d44002a0d00000a0000000d0a00002a2a0000d3
:102d54002a2a00002a2000005553000042200000c7
:102d640045720000726f0000722000002d200000e8
:102d7400636100006e6e00006f7400002065000047
:102d84006e7500006d6500007261000074650000de
:102d9400206400006576000069630000652000007f
:102da4002a2a00002a2a00002a0d00000a00000036
:102db4000d0a00002a2a00002a2a00002a20000006
:102dc400555300004220000045720000726f00005d
:102dd400722000002d200000636c00006965000073
:102de4006e740000206400007269000076650000c3
:102df40072200000696e00006974000069610000bf
:102e04006c6900007a610000746900006f6e000054
:102e140020650000727200006f720000202a00001a
:102e24002a2a00002a2a00000d0a0000000d0000d2
:102e34000a2a00002a2a00002a2a0000205500003d
:102e44005342000020450000727200006f720000bf
:102e5400202d0000206f000075740000206f00001a
:102e6400662000006865000061700000206d0000ad
:102e7400656d00006f720000792000002a2a0000ae
:102e84002a2a00002a0d00000a0000000d0a000092
:102e94002a2a00002a2a00002a2000005553000094
:102ea4004220000045720000726f00007220000092
:102eb4002d200000756e0000737000006563000033
:102ec4006966000069650000642000002a2a000089
:102ed4002a2a00002a0d00000a00000044650000b0
:102ee40076690000636500002044000065740000fa
:102ef4006163000068650000642000000045000074
:102f0400787000006c6f0000726500007231000080
:102f140036200000426f000061720000640000006f
:102f24005553000042200000484900004448000076
:102f34006f73000074200000446500006d6f000092
:102f44000000000048490000443a0000204400000a
:102f5400657600006963000065200000617400006c
:102f64007461000063680000656400002e0d0000b9
:102f74000a00000030310000323300003435000014
:102f84003637000038390000414200004344000055
:102f9400454600000a0d000045720000726f0000f3
:0c2fa400723a0000202000000000000035
:020000040000fa
:102fb0000600fa0020479800314798005181200010
:102fc000914078002e40900080cf500003003200e6
:102fd000600020002007980019003700a0488000fa
:102fe000000f7800120037001e007800c0589000d3
:102ff0003e40900080cf50000b003a009e007800c9
:10300000214090000030a100a04098009e00780070
:10301000214090000040a100a04098000000eb007b
:1030200020079800060037001e007800100f780077
:103030001e00e000ecff3a0040012000200798004d
:103040002e0090000080fa00000006001000fa0038
:10305000004f7800114798002247980023079800f6
:10306000340798004507980056079800474f980086
:1030700015c8bf009e4f50000300320060002000c2
:103080007007980053003700e140800000f02000f6
:103090008080600000402000808f500003003200dc
:1030a00011002000710798004a003700a0488000f6
:1030b000a040900000c8b30000c060000004e00021
:1030c00003003a000001200070079800410037001b
:1030d0002e409000eb4f500002003a000040eb0001
:1030e000180e07002e409000e14f500005003a00f6
:1030f0002e0090000000e00002003a003e00900028
:10310000100e0700b04880009e40900001487800f3
:10311000b04880000000e800ae4090000148780010
:10312000b04880008080e8002e0090008048780041
:10313000b0488000e30040002e0090004800de0010
:1031400080487800b0488000e40040003e009000d5
:1031500080487800b0488000e50040003e009000c4
:103160004800de0080487800b0488000e60040005b
:103170004e00900080487800b0488000e700400092
:103180004e0090004800de00804878004e489000d5
:103190000004e00007003a00b1488000a048800029
:1031a0004e029000de01900082002000330b0700e9
:1031b00006003700b1488000a04880004e02900011
:1031c000de01900082002000ee0a07000000eb0004
:1031d000700798007e0090000080fa000000060052
:1031e0000400fa00004f7800e040800001f0200069
:1031f000010060000000e00003003a00100320001e
:10320000100798001d003700e140800000f020000a
:103210008080600000402000808f50000b003a004a
:10322000e0408000010f200001006000f00f50001e
:1032300003003a00a0032000100798000f00370099
:1032400000032000100798000c003700e1408000c8
:1032500000f020008080600000502000808f50002f
:1032600004003a0016c8bf000080fb001007980059
:103270000200370020032000100798001e00900075
:103280000080fa00000006000600fa00008fbe0071
:10329000a04880000000e0000d003a00200220005d
:1032a000a6fd0700a0488800a04880000000e000bc
:1032b00003003a000000eb002007980012003700de
:1032c000a14880000000eb00800878000100370072
:1032d0008c0a0700a0488000304088000000eb0006
:1032e000e04088000080eb00f04088000040eb00e8
:1032f00014e8b7000040eb0015e8b7002008a8006c
:1033000010002000200798002e0090000080fa0096
:10331000000006000c00fa00204798003147980092
:103320002207980034079800450798005181200033
:10333000914078002e40900080cf50000300320072
:10334000600020005007980047003700e1408000ef
:1033500000f020008080600000402000808f50003e
:103360000300320010002000500798003e00370094
:10337000a0488000000f7800370037001e0078005a
:10338000c05890003e40900080cf500030003a007e
:103390001e007800e00890000030200000806000ef
:1033a0000000e00003003a00800120005007980070
:1033b0002d0037001e007800405890000004e00007
:1033c0000300350050012000500798002600370008
:1033d0001e00780020409000684060000004e0007b
:1033e0000300320010012000500798001e00370033
:1033f0001e00780020409000704060000004e00053
:10340000030032002001200050079800160037000a
:103410001e007800a040900000c8b30000c060000b
:103420000004e00003003a0000012000500798006b
:103430000d0037003e019000ae0090001e007800a5
:10344000d30a07000000eb00500798000600370081
:103450001e007800100f78001e00e000c7ff3a0041
:1034600040012000500798005e0090000080fa00a4
:10347000000006000400fa00004f780015c8bf00e5
:103480009e4f50000300320060002000100798009b
:103490000c003700e040800001f0200001006000d7
:1034a0000000e00003003a00300020001007980000
:1034b000040037000000eb00e04088000000eb0053
:1034c000100798001e0090000080fa00000006001f
:1034d0000400fa00004f780015c8bf009e4f50004e
:1034e0000300320060002000100798000c00370035
:1034f000e140800000412000808f50000300320036
:10350000300020001007980005003700e0408000e0
:103510000000e800e04088000000eb001007980081
:103520001e0090000080fa00000006000400fa006f
:10353000004f78001147980015c8bf009e4f5000fb
:1035400003003200600020001007980015003700cb
:10355000e140800000f020008080600000402000fa
:10356000808f5000030032001000200010079800e8
:103570000c003700de0d07000000e0000300320001
:103580002000200010079800060037001e40900021
:1035900012e8b70000332000e04088000000eb0094
:1035a000100798001e0090000080fa00000006003e
:1035b0000200fa000000eb004024880015c8bf009c
:1035c0000004e0000d0032000040eb00004f7800e6
:1035d00015c8bf0024002000050020000e0178005f
:1035e000e1002000a120070015c8bf001300200043
:1035f0005281200071002000ed0a07006000b80031
:1036000021ff07000080fa00000006000400fa0015
:10361000004f780015c8bf009e4f500003003200d5
:1036200060002000100798000c003700e140800087
:1036300000402000808f5000030032003000200046
:1036400010079800050037009404a90000412000ed
:10365000e04088000000eb00100798001e0090007a
:103660000080fa00000006002a00fa00881f780097
:10367000f0408000e10f400004003200f040800084
:10368000e04088000080eb00f0408800e0408000cf
:1036900001f0200001006000401798000020200089
:1036a000ce109000808f5000520232000020200087
:1036b000ce109000808f500008003e004e10900009
:1036c0000000e0001200320000102000ce10900038
:1036d000808f5000a6003200950537000040200082
:1036e000ce109000808f500007053200005020005f
:1036f000ce109000808f5000400532000030200036
:10370000ce109000808f500099023200880537005b
:10371000e1408000000f2000808060003117980099
:103720003e109000f00f50005d00320000022000bb
:10373000be109000808f5000630032003e10900059
:103740000000e000010032007905370098ff070013
:10375000a14880000000eb0080087800a1488000ac
:103760000000eb0090009800a148800031409000dc
:103770000000a000b0409800a148800021409000c7
:103780000070a000a0409800a14880000004200024
:10379000c0009800a24880006000b80000099800ae
:1037a00011099800a14880000040eb00c058980023
:1037b000a14880000040eb0080589800a14880009c
:1037c000610890000080a1000090a100e00898002e
:1037d000a14880000000eb00d008980030c0b30082
:1037e00002e8b7000040eb0012e8b7000040eb0031
:1037f00013e8b7000040eb0014e8b7000000eb004e
:10380000d04088000000eb0060248800f00f20000a
:10381000502488000000eb0010248800f00f2000e6
:10382000002488000000eb0080248800f00f2000b6
:10383000702488008cc4a80000a020004800de008e
:10384000c024880080002000a0248800a000200060
:10385000a024880080002000a0248800c00320004d
:103860003024880020012000302588000000eb0073
:10387000402588000000eb00b0248800aae4a900dd
:10388000a004200000258800e140800000ff200007
:103890000080600070004000e04088002405370090
:1038a00020c8bf00614060000004e0002005320035
:1038b000e140800000ff20000080600070004000b8
:1038c000e04088001a053700e80047000040eb00a0
:1038d00080487800e800470020c3b300904098007b
:1038e000680147002400200005002000d1002000ce
:1038f00000c0eb00dd1f07000000e00018003200f0
:10390000100020004024880071048000f0fb2f008c
:10391000008060007004880071068000f00f2f00a6
:103920000080600070068800710680000060200042
:103930000080700070068800f10480000004200000
:1039400000807000f0048800e140800000ff20004b
:103950000080600070004000e0408800f404370000
:103960002008a90000012000e0408800f004370092
:10397000e0408000010f2000010060002017980047
:1039800000022000ae109000808f5000b000320086
:1039900000022000ae109000808f500007003e0013
:1039a0002e1090000000e0000d003200ae109000dc
:1039b000f08f500029003200dd04370000032000a2
:1039c000ae109000808f50002901320000042000ca
:1039d000ae109000808f50007f013200d404370079
:1039e000e04080006f006000101798001e109000eb
:1039f000e10f5000ce0432009e109000e18f500085
:103a0000040039001e109000e20f50000d0032003b
:103a1000c704370010002000502488008c04a80040
:103a2000b00f2000204088000004200000248800ff
:103a300082c4a800e04080000000e800e040880068
:103a4000bb043700e140800000ff200000806000e0
:103a500070004000e0408800b5043700e04080007e
:103a60006f006000001798008e109000e28f5000e9
:103a7000620032000e109000e20f500004003e0081
:103a80008e1090000100e00008003200a80437000a
:103a90000e109000e30f5000a50432008e1090002d
:103aa000e48f500060003200a1043700b04880006d
:103ab0000000e00004003200b0488000f1fb070085
:103ac0000000eb00b0488800800020009bfb07004e
:103ad000b0488800b04880000000e00005003a00cf
:103ae00030c3b30016e8b70000502000e040880063
:103af0008f0437000040eb0012e8b7000040eb00f5
:103b000013e8b7000000eb00d040880030c0b300dd
:103b100001e8b700d0002000502588000000eb002d
:103b2000602588000000eb00702588000000eb0095
:103b3000802588000000eb00902588000000eb0045
:103b4000a02588000000eb00b02588000000eb00f5
:103b5000c02588000000eb00d02588000000eb00a5
:103b6000e02588000000eb00f02588000000eb0055
:103b7000002688000000eb00102688000000eb0003
:103b8000202688000000eb00302688000000eb00b3
:103b900040268800414920009140780000c8b300c9
:103ba00000c060000004e00006003a001a08a80007
:103bb00000c8b30014e8b70000082000b024880053
:103bc000aae4a8009424a8009424a9001a88a900b3
:103bd0001aa8a9009484a80030032000204088007f
:103be000000420000024880082c4a800e040800077
:103bf0000000e800e04088004d0437009484a900ec
:103c00009404a800b0002000204088000004200098
:103c10000024880082c4a800e04080000000e80082
:103c2000e040880042043700f00020006024880053
:103c3000f00f200080248800e140800000ff200079
:103c40000080600070004000e040880038043700c9
:103c5000e04080006f006000700f98007e089000c8
:103c6000e10f500039003200fe089000e18f500053
:103c7000040039007e089000e20f50004e00320030
:103c80002b043700904880000000e0000400320060
:103c9000904880007bfb07000000eb009048880004
:103ca000b148800000c8b30080487800b048800068
:103cb0008000e80060c0b30080487800b048800011
:103cc0008080e8000040eb0080487800b048800029
:103cd000e300400010c0b30080487800b048800086
:103ce000e40040000040eb0080487800b0488000cd
:103cf000e50040000040eb0080487800b0488000bc
:103d0000e600400080c0b30080487800b0488000e2
:103d1000e70040000040eb0080487800b048800099
:103d2000b1488000a5488000840020008001780010
:103d3000820020000500780012080700e0408000a3
:103d40000000e800e0408800f9033700a048800048
:103d5000a040900000c8b30000c060000004e00074
:103d6000f3033200a0488000204090000044b200dd
:103d70000004e0000e003200b04880006400400003
:103d800010407800e94f500005003a0050c3b300de
:103d900016e8b70000502000e0408800e403370038
:103da000e04080000000e800e0408800e0033700c9
:103db000cc040700de033700b048800010407800d4
:103dc0000080fb00ddfa07009048880090488000e2
:103dd0000000e00005003a0030c3b30016e8b70069
:103de00000502000e0408800d10337009148800057
:103df000b04880001040780080487800a1488000da
:103e0000b0488000704090000080fb00c000980027
:103e1000b04880001bfb07000000eb00b0488800a2
:103e2000a048800040009000c4fa0700b048880015
:103e3000b04880000000e00005003a0030c3b30045
:103e400016e8b70000502000e0408800b8033700b3
:103e500030c0b30001e8b700e140800000ff20005f
:103e60000080600070004000e0408800b003370030
:103e7000e04080006f006000600f9800ee08900046
:103e8000e18f50003b0032006e089000e10f5000bf
:103e900004003900ee089000e28f50004600320026
:103ea000a303370094c4bf000042b2000004e00046
:103eb0009f033a00b148800000c8b30080487800f2
:103ec000b04880008000e80060c0b30080487800ff
:103ed000b04880008080e8000040eb008048780017
:103ee000b0488000e300400010c0b3008048780074
:103ef000b0488000e40040000040eb0080487800bb
:103f0000b0488000e50040000040eb0080487800a9
:103f1000b0488000e60040009048800010407800e3
:103f200080487800b0488000e70040000040eb0087
:103f30008048780090488000104078000080fb00a6
:103f400091488000b5488000a648800000027800b3
:103f5000810178008200200085007800060078004a
:103f600088070700e04080000000e800e04088008b
:103f70006f033700a0488000a040900000c8b30045
:103f800000c060000004e00069033200a048800027
:103f9000204090000044b2000004e0000400320021
:103fa000e04080000000e800e04088006003370047
:103fb0004c0407005e03370030c0b30001e8b700cf
:103fc000e140800000ff20000080600070004000a1
:103fd000e040880056033700a4040700e140800059
:103fe00000f02000008060000010b000e040880079
:103ff0004f033700e0408000010f20000100600007
:104000000000e0000100320049033700e04080007a
:104010006f006000500f98005e089000e10f5000a4
:1040200032003200de089000e18f500004003900b9
:104030005e089000e20f50003d0032003c03370064
:1040400010c0b30015e8b700b14880000040eb0095
:1040500080487800b04880008000e80050c0b3007d
:1040600080487800b04880008080e80015c8bf0014
:1040700080487800b0488000e30040000040eb003a
:1040800080487800b0488000e40040000040eb0029
:1040900080487800b0488000e50040000040eb0018
:1040a00080487800b0488000e60040000040eb0007
:1040b00080487800b0488000e70040000040eb00f6
:1040c00080487800b1488000a04880000002eb00e2
:1040d0008001eb008200200068070700e0408000bc
:1040e0000000e800e040880011033700a04880008d
:1040f000a040900000c8b30000c060000004e000d1
:104100000b033200a0488000204090000044b20021
:104110000004e00004003200e04080000000e800fd
:10412000e040880002033700ee0307000003370079
:104130001ac8bf00614060000080fb004700dd003e
:104140008040780015c8bf0000c0700014e8b700b8
:1041500030c0b30001e8b700e140800000f020006b
:10416000008060000010b000e0408800f0023700de
:10417000e0408000010f200001006000400f980027
:1041800000022000ce089000808f5000c400320052
:1041900000022000ce089000808f500007003e00f3
:1041a0004e0890000000e0000d003200ce089000a4
:1041b000f08f500021003200dd02370000032000a4
:1041c000ce089000808f50002201320000042000b1
:1041d000ce089000808f5000bc013200d40237001e
:1041e000904880001050900000e8b7000a003700a7
:1041f0007048800010009000100798007048800000
:10420000100078001ffa0700704880001dfa0700b0
:104210001e00900070488800704880000000e00098
:10422000f3ff3a00e140800000ff200000806000c2
:1042300070004000e0408800bd023700e040800090
:104240006f006000300f98003e089000e10f5000b2
:1042500033003200be089000e18f500004003900a6
:104260003e089000e20f50003e003200b0023700de
:10427000b148800000c8b30080487800b048800092
:104280008000e80060c0b30080487800b04880003b
:104290008080e80000c8bf000040e9008048780046
:1042a000b0488000e300400020c0b30080487800a0
:1042b000b0488000e40040000040eb0080487800f7
:1042c000b0488000e50040000040eb0080487800e6
:1042d000b0488000e600400080c0b300804878000d
:1042e000b0488000e70040000040eb0080487800c4
:1042f000b0488000b1488000a548800084002000bc
:104300008001780082002000050078009d060700eb
:10431000e04080000000e800e040880084023700b0
:10432000a0488000a040900000c8b30000c060001a
:104330000004e0007e023200a0488000204090008f
:104340000044b2000004e00004003200e0408000bd
:104350000000e800e04088007502370061030700b4
:10436000730237006000200074f9070010079800fe
:104370001e0090000000e00005003a0030c3b300ca
:1043800016e8b70000502000e040880068023700bf
:104390001e049000b0488000630040001040780088
:1043a0000080fb00c800dd00b04880000080e8000d
:1043b000104078000080fb00008040005ff907009b
:1043c000000c7800180078000000e00009003a00b6
:1043d0001e009000abf907000000eb0010079800ea
:1043e00030c3b30016e8b70000502000e04088005a
:1043f0004f0237001e009000100078000001780086
:10440000b048800063004000104078000080fb004e
:10441000c800dd00b04880000080e800104078004f
:104420000080fb0080814000f00f20008080610050
:1044300022409000604060000140700020419800e0
:10444000c818de00324090006040600001407000fb
:10445000304198009e0090007048800090009800c5
:104460001e009000704888001e0090001000780028
:10447000804888009e00900000c8bf00c04098009f
:1044800030c0b30001e8b700e140800000ff200029
:104490000080600070004000e04088002402370087
:1044a000e04080006f006000200f9800ae08900090
:1044b000e18f5000450032002e089000e10f5000bf
:1044c00004003900ae089000e28f50005000320026
:1044d00017023700b148800000c8b3008048780058
:1044e000b04880008000e80060c0b30080487800d9
:1044f000b04880008080e80000c8bf000040e900ac
:1045000080487800b0488000e300400020c0b3003d
:1045100080487800b0488000e40040000040eb0094
:1045200080487800b0488000e50040000040eb0083
:1045300080487800b0488000e60040007048800065
:10454000100078000080e800104078008048780073
:10455000b0488000e70040007048800010007800fc
:104560006300400010407800804878007048800068
:104570001000780080007800214090000081fb004e
:10458000314090000080fb004800dd000200700018
:10459000800078007048800010007800b5488000e6
:1045a000a648800001027800800178008200200087
:1045b0008500780006007800f2050700e0408000e2
:1045c0000000e800e0408800d9013700a0488000e2
:1045d000a040900000c8b30000c060000004e000ec
:1045e000d3013200a0488000204090000044b20077
:1045f0000004e00004003200e04080000000e80019
:10460000e0408800ca013700b6020700c801370041
:1046100030c0b30001e8b70000c8bf000040e900a7
:1046200000e8b70000c8bf000004e000030032004b
:1046300000312000e0408800bd013700e1408000eb
:1046400000ff20000080600070004000e040880013
:10465000b7013700e04080006f006000100f980045
:104660001e089000e10f5000420032009e089000aa
:10467000e18f5000070039001e089000e20f500043
:10468000790032009e089000e38f500087003200ce
:10469000a70137007605070012c8bf000004e0003c
:1046a00011003a0070488000300798000a00370077
:1046b0003e0090001000780080488800180707002e
:1046c0000000e0001f003a00690507003e0090006e
:1046d00090009000310798003e0090000000e0003c
:1046e000f3ff3a0017003700704880003007980049
:1046f000030037003e0090009000900031079800c2
:104700003e0090000000e000050032003e009000f6
:10471000c040900012c8bf0080cf5000f5ff3a00a3
:104720003e0090001000780080488800fc060700da
:104730000000e00003003a004d0507000000eb0018
:10474000300798003e0090000000e00005003a00ad
:1047500040c3b30016e8b70000502000e0408800d6
:1047600073013700e04080000000e800e04088006e
:104770006f0137001ac8bf00644060000004e00009
:1047800033003a001a48a800b14880000040eb000e
:1047900080487800b04880008000e80030c0b30056
:1047a000804878001ac8bf00684060000004e0003c
:1047b00005003200b04880008080e80030c0b300bf
:1047c0008048780004003700b04880008080e8000e
:1047d00040c0b30080487800b0488000e30040004b
:1047e0000040eb0080487800b0488000e4004000c2
:1047f0000040eb0080487800b0488000e5004000b1
:104800000040eb0080487800b0488000e60040009f
:104810000040eb0080487800b0488000e70040008e
:104820000040eb0080487800b1488000a04880003c
:104830000002eb008001eb00820020008f050700e2
:10484000e04080000000e800e040880038013700c8
:10485000e140800000ff2000008060007000400008
:10486000e040880032013700a0488000a04090005e
:1048700000c8b30000c060000004e0002c0132005a
:10488000a0488000204090000044b2000004e000f6
:1048900004003200e04080000000e800e0408800b2
:1048a000230137000f0207002101370030c0b30099
:1048b00001e8b700e140800000ff200000806000b8
:1048c00070004000e040880019013700e04080009f
:1048d0006f006000000f98000e089000e10f50007c
:1048e000330032008e089000e18f5000070039003d
:1048f0000e089000e20f50003e0032008e0890003b
:10490000e38f50004100320009013700b1488000b8
:104910000040eb0080487800b04880008000e8004c
:1049200090c0b30080487800b04880008080e800e4
:1049300012c8bf0080487800b0488000e300400003
:104940000040eb0080487800b0488000e400400060
:104950000040eb0080487800b0488000e50040004f
:104960000040eb0080487800b0488000e60040003e
:104970000040eb0080487800b0488000e70040002d
:104980000040eb0080487800b1488000a0488000db
:104990000002eb008001eb008200200037050700d9
:1049a000e04080000000e800e0408800e0003700c0
:1049b000a0488000a040900000c8b30000c0600084
:1049c0000004e000da003200a0488000204090009f
:1049d0000044b2000004e00004003200e040800027
:1049e0000000e800e0408800d1003700bd0107006a
:1049f000cf00370030c0b30001e8b700e0408000ce
:104a00000000e800e0408800c9003700e140800075
:104a100000f02000008060000010b000e04088003e
:104a20001ac8bf000044b2000004e00016003200c3
:104a300017c8bf00004f78001e80fb00c300dd00d8
:104a4000a08d200000804000100278001e80fb0036
:104a50004300dd00e4004000a08d20000080400005
:104a60001001be0015c8bf00040001000000e000f6
:104a7000af003a0090c3b30016e8b7000050200022
:104a8000e0408800aa003700c14880002107980054
:104a9000190037002e009000c0409000014f7800b0
:104aa0001e80fb00c300dd00a08d200000804000c0
:104ab000100278001e80fb004300dd00e40040008f
:104ac000a08d2000008040001001be0015c8bf006e
:104ad000040001000000e00004003a0090c3b300ad
:104ae00016e8b70000502000e04088002e0090003b
:104af00090007800210798002e0090000000e00050
:104b0000e4ff3a008a003700e1408000000f2000f7
:104b100080806000710798007e0090000000e00037
:104b200083003200fe009000f08f50000100320040
:104b30007f003700e04080006f0060006007980051
:104b40006e009000e20f500079003200ee009000fd
:104b5000e28f500007003e006e0090000000e00071
:104b600073003200ee009000e18f50000b00320025
:104b70006f0037006e009000e40f50006c003200b0
:104b8000ee009000e48f50000e0039006e0090009f
:104b9000e50f500016003200650037009444a8006d
:104ba00050012000204088000004200000248800dc
:104bb00082c4a800e04080000000e800e0408800d7
:104bc0005b0037009444a9009404a800b0002000c2
:104bd00020408800000420000024880082c4a8002f
:104be000e04080000000e800e0408800500037000e
:104bf00000402000e04088004d003700e040800089
:104c0000010f2000010060000000e0000100320000
:104c10004700370080002000a02488000000eb003f
:104c200060248800f00f2000502488000000eb0072
:104c300010248800f00f2000002488000000eb0002
:104c400080248800f00f2000702488008c04a800c5
:104c500016c8bf000080fb005007980040032000ea
:104c6000de009000808f50001800320040032000ca
:104c7000de009000808f500008003c005e00900035
:104c8000e70f50001400320030032000de009000d7
:104c9000808f5000160032001800370050032000ab
:104ca000de009000808f500005003200900320004d
:104cb000de009000808f50000a0032000f003700a5
:104cc00080c0b300004f78000e00370000c1b30071
:104cd000004f78000b00370010c1b300004f780080
:104ce0000800370020c1b300004f780005003700ee
:104cf00030c1b300004f78000200370040c1b3005c
:104d0000004f78009e80fb0015c8bf0014002000f3
:104d10000500200082812000d41a0700e1408000b5
:104d200000ff20000080600070004000e04088002c
:104d30004f0478000080fa00000006000400fa002a
:104d40002047980031479800518120009140780019
:104d50002e40900080cf500015003a00a0488000ff
:104d6000000f7800100037001e007800c058900037
:104d70003e40900080cf500009003a009e0078002d
:104d8000214090000050a000a04098009e007800b4
:104d9000214090000070a000a0409800040037005f
:104da0001e007800100f78001e00e000eeff3a00b1
:104db0000080fa00000006000c00fa00404798004e
:104dc000514798003207980043079800518120000e
:104dd000914078004e40900080cf50000900320092
:104de000be00900060c0b300804878004e01900083
:104df0006000b8000089be00100020005007980035
:104e00003f003700a14880001107980034003700a8
:104e10001e009000c05890005e40900080cf50006f
:104e20002c003a001e009000204090000080fb0003
:104e30004700de00004f78001e00900020409000e8
:104e40000044b2000004e00009003200be009000ff
:104e50000040eb00804878001e0090009008900011
:104e6000000890004e0190000089be001600370037
:104e70001e00900020409000684060000004e000a8
:104e800004003200be00900010c1b30080487800da
:104e90000d0037001e009000204090007040600020
:104ea0000004e000050032001e009000e058900071
:104eb0003e0090000148780003003700be009000db
:104ec00090c1b300804878001e80fb005007980016
:104ed0000b0037001e00900090007800110798002a
:104ee0001e0090000000e000c9ff3a00be009000e4
:104ef00040c1b3008048780010002000500798009f
:104f00005e0090000080fa00000006000600fa0033
:104f1000000f780021479800324798002e409000fb
:104f2000e14f400012003a003e4090000004e000d3
:104f30000f003a00c00020009e0f100005003a004c
:104f40009bf907002008a9000000eb00200798004b
:104f500009003700f00020009e0f100004003a0006
:104f60002008a8000000eb0020079800020037008e
:104f700030002000200798002e0090000080fa00ea
:104f8000000006000c00fa00204798003147980006
:104f900022079800340798004507980051812000a7
:104fa000914078002e40900080cf500003003200e6
:104fb000600020005007980047003700e140800063
:104fc00000f020008080600000402000808f5000b2
:104fd0000300320010002000500798003e00370008
:104fe000a0488000000f7800370037001e007800ce
:104ff000c05890003e40900080cf500030003a00f2
:105000001e007800e0089000003020000080600062
:105010000000e00003003a008001200050079800e3
:105020002d0037001e007800405890000004e0007a
:1050300003003d0050012000500798002600370073
:105040001e00780020409000684060000004e000ee
:105050000300320010012000500798001e003700a6
:105060001e00780020409000704060000004e000c6
:10507000030032002001200050079800160037007e
:105080001e007800a040900000c8b30000c060007f
:105090000004e00003003a000001200050079800df
:1050a0000d0037003e019000ae0090001e00780019
:1050b000fb0307000000eb005007980006003700d4
:1050c0001e007800100f78001e00e000c7ff3a00b5
:1050d00040012000500798005e0090000080fa0018
:1050e000000006000000fa003140800021409000de
:1050f0000040a100a0409800314080002140900075
:105100000030a100a040980001c8bf000040e900a5
:1051100001e8b70001c8bf000004e000050032004c
:10512000e040800001ff2f0001006000e0408800a7
:105130000d00370002c8bf000040e90002e8b700d8
:1051400002c8bf000004e00003003200001120008c
:10515000e04088000400370070c0b30016e8b700d4
:1051600000502000e04088000080fa0000000600a7
:105170000a00fa00204798003147980042479800fb
:10518000330798000000eb00000f78002f00370075
:105190001e0078004300dd00e6004000a08e2000e5
:1051a00000804000100078000000d10061406000e5
:1051b000e14f500024003a001e007800c300dd00db
:1051c000a08e200000804000904078002e4090008b
:1051d00080cf50001c003a001e007800c300dd00a4
:1051e000a08e200000804000904090003e40900043
:1051f00080cf500014003a001e0078004300dd000c
:105200008080e800a08e2000008040009040780060
:105210004e40900080cf50000b003a001e007800f6
:105220004300dd00e4004000a08e2000008040002c
:10523000904090003e00900001487800100020004f
:1052400040079800060037001e0fe80010002000fd
:105250009e0f1000ceff34000000eb0040079800c6
:105260004e0090000080fa00000006000600fa00e0
:1052700090488000000f78000000eb0010079800b5
:105280001ac8a900680037001e0090004300dd0026
:10529000e6004000a08e2000008040001000780052
:1052a0000000d100614060000004e0001e003200f8
:1052b0001e009000c300dd00a08e20000080400092
:1052c000904078001e0078004040900080cf500051
:1052d00033003a001e009000c300dd00a08e2000c5
:1052e00000804000904090001e00780050409000e8
:1052f00080cf50002a003a001e0090004300dd00dd
:105300008080e800a08e200000804000904078005f
:105310001e0078006040900080cf500020003a00ce
:105320001ac8a8001e0037001e009000c300dd0050
:10533000a08e200000804000900178009e00780040
:10534000014890000081fb00114890000080fb00a4
:105350004800dd0002007000808f510010003a000c
:105360001e0090004300dd008080e800a08e200039
:1053700000804000900178009e0078002148900055
:105380000081fb00314890000080fb004800dd00f8
:1053900002007000808f510001003a001ac8a80076
:1053a0001ac8bf000044b2000004e0001b00320035
:1053b0001e0090004300dd00e4004000a08e2000ad
:1053c000008040001040900017e8b7001e009000d9
:1053d0004300dd00e6004000a08e20000080400079
:1053e000100078004200de00614060000004e00030
:1053f000070032001e0090004300dd00e400400082
:10540000a08e2000008040001040780012e8b70015
:105410001000200020079800080037001e009000b0
:105420000000e800100798001e009000e10f5000f7
:1054300095ff36000000eb00200798002e0090003a
:105440000080fa00000006000600fa0020479800dd
:1054500031479800c0488000000f78000d003700e9
:105460001e007800a04090002e40900080cf500099
:1054700008003a001e007800b04090003e409000c6
:1054800080cf500003003a001e00780020079800eb
:10549000040037001e00e000f1ff3a000000eb00be
:1054a000200798002e0090000080fa0000000600ff
:1054b0001200fa000000eb00000f7800e0408000ce
:1054c00094c4bf000042b2000004e000e6013a00cc
:1054d0008080200010407800614060000004e000ff
:1054e0003b013a00a04880001007980031013700c6
:1054f0001e009000e0089000003020000080600056
:105500000000e00028013a001e009000a04090003a
:1055100000c8b30000c060000004e00022013a00af
:105520001e009000304088001e009000005890003f
:105530008080fb00000f200080806000010f980039
:10554000000220008e089000808f5000550032002d
:10555000000320008e089000808f5000ac003200c5
:105560000e089000f00f50000100320003013700d8
:105570001e009000005890000080fb006f0060004b
:1055800070079800fe009000e18f50001d0032006f
:105590007e009000e10f500004003c00fe009000ef
:1055a0000100e000080032003b0037007e00900060
:1055b000e20f500028003200fe009000ef8f5000f4
:1055c0002d0032003400370031408000314090001f
:1055d0000010a100b0409800d0c0b3001a05070029
:1055e0001e00900040589000d1c0b300ec040700aa
:1055f00081802000114078000000a00080487800e1
:1056000099013700324080003040800090089000bf
:10561000000890005001980061019800314080001e
:10562000314090000010a000b040980090c0b3003e
:10563000050507001e0090004058900091c0b3007f
:10564000d704070081802000114078000000a000ee
:1056500080487800840137009e0090000040eb00f5
:10566000805898009e009000214090000070a0009b
:10567000a0409800c30037009e0090000040eb005f
:10568000805898009e009000214090000070a0007b
:10569000a0409800bb00370010002000000f7800e9
:1056a000b80037001e009000005890000080fb00fa
:1056b0006f006000600798006e009000e20f5000dd
:1056c0002b003200ee009000e28f500007003c00fb
:1056d0006e0090000000e0000b003200ee00900031
:1056e000e18f500017003200460037006e00900036
:1056f000e30f500033003200ee009000ef8f5000b7
:10570000380032003f0037003140800031409000c7
:105710000010a100b0409800d0c0b300ca04070038
:105720001e00900040589000d1c0b3009c040700b8
:1057300081802000114078000000a000804878009f
:105740004901370090c0b300bf0407001e0090005d
:105750004058900091c0b300910407008180200060
:10576000114078000000a000804878003e0137001a
:105770003240800030408000900890000008900087
:105780005001980061019800314080003140900044
:105790000010a000b040980010c0b300aa04070099
:1057a0001e0090004058900011c0b3007c04070018
:1057b00081802000114078000000a000804878001f
:1057c000290137009e0090000040eb0080589800af
:1057d0009e009000214090000070a000a040980022
:1057e000680037009e0090000040eb008058980051
:1057f0009e009000214090000070a000a040980002
:105800006000370010002000000f78005d003700b6
:105810001e009000005890000080fb006f006000a8
:10582000500798005e009000e20f50002b003200fd
:10583000de009000e28f500007003c005e00900008
:105840000000e0000b003200de009000e18f50000d
:1058500017003200460037005e009000e30f500052
:1058600033003200de009000ef8f5000380032002d
:105870003f00370031408000314090000010a1000f
:10588000b0409800d0c0b3006f0407001e00900025
:1058900040589000d1c0b30041040700818020002f
:1058a000114078000000a00080487800ee0037002a
:1058b00010c0b300640407001e0090004058900020
:1058c00011c0b30036040700818020001140780029
:1058d0000000a00080487800e300370032408000dc
:1058e000304080009008900000089000500198001f
:1058f0006101980031408000314090000010a0000c
:10590000b040980090c0b3004f0407001e00900004
:105910004058900091c0b30021040700818020000e
:10592000114078000000a00080487800ce003700c9
:105930009e0090000040eb00805898009e00900070
:10594000214090000070a000a04098000d0037009a
:105950009e0090000040eb00805898009e00900050
:10596000214090000070a000a04098000500370082
:1059700010002000000f7800020037001000200007
:10598000000f78001e00e000070032009e0090002b
:105990000040eb00805898009e009000214090004d
:1059a0000070a000a04098001e00900090007800b9
:1059b000110798001e0090000000e000ccfe3a00a5
:1059c00081802000114078000000a000804878000d
:1059d0008080200010407800624060000004e000f9
:1059e000a1003a00a04880001007980097003700f7
:1059f0001e009000e00890000030200080806000d1
:105a000000302000808f50008d003a001e00900072
:105a1000a040900000c8b30000c060000004e00097
:105a2000090032001e009000300090000000e000ed
:105a300083003a001e009000a00090001e0090001d
:105a4000310098007e0037001e0090003040880032
:105a50001e009000005890008080fb00000f200086
:105a6000808060004107980000042000ce00900074
:105a7000808f50000500320000052000ce0090000d
:105a8000808f500032003200620037001e0090000c
:105a9000005890000080fb006f0060003007980005
:105aa0003e009000e10f500016003200be00900052
:105ab000ef8f50001b0032003e0090000000e0001d
:105ac000010032001f0037001e00900030009000df
:105ad0000000e00051003a001e009000a00090007d
:105ae0001e0090003100980090c0b300d60307005c
:105af0001e0090004058900091c0b300a80307001a
:105b0000590037009e0090000040eb00805898003c
:105b10009e009000214090000070a000a0409800de
:105b20003e0037009e0090000040eb008058980037
:105b30009e009000214090000070a000a0409800be
:105b40003600370010002000000f780033003700c7
:105b50001e009000005890000080fb006f00600065
:105b600020079800ae009000e18f50001600320030
:105b70002e009000ef0f50001b003200ae0090008e
:105b80000100e000010032001f0037001e009000fd
:105b9000300090000000e00020003a001e0090005d
:105ba000a00090001e0090003100980010c0b300cb
:105bb000a50307001e0090004058900011c0b300dc
:105bc00077030700280037009e0090000040eb009c
:105bd000805898009e009000214090000070a00026
:105be000a04098000d0037009e0090000040eb00a0
:105bf000805898009e009000214090000070a00006
:105c0000a04098000500370010002000000f780029
:105c10000200370010002000000f78001e00e00096
:105c2000070032009e009000214090000070a0000c
:105c3000a04098009e0090000040eb008058980023
:105c40001e00900090007800110798001e00900040
:105c50000000e00066ff3a008180200011407800db
:105c60000010a000804878000080fa0000000600c4
:105c70000200fa0007003700c048800010007800da
:105c8000000f7800c04880007ef307001e007800f7
:105c9000c0488800c04880000000e000f6ff3a00dd
:105ca000a04880000000e000120032000a00370027
:105cb000a04880001000780010007800000f7800e5
:105cc000a0488000100078006ef30700a148800013
:105cd0001e00780080087800a0488000100078003e
:105ce0000000e000f2ff3a00a14880000000eb0055
:105cf00080087800a0488000304088000080fa00ca
:105d0000000006000200fa000a0037007048800018
:105d100010009000000f780070488000100078009c
:105d200058f307007048800056f307001e00780003
:105d300070488800704880000000e000f3ff3a00df
:105d4000904880000000e00004003200904880008d
:105d50004cf307000000eb0090488800b04880003a
:105d60000000e00004003200b048800045f3070066
:105d70000000eb00b0488800bdff07000080fa007b
:105d8000000006000a00fa00000f780011079800d2
:105d90002207980033079800440798009e00780077
:105da000214090000030a100a04098009e007800a3
:105db000214090000040a100a04098009e00780083
:105dc000214090000050a100a04098009e00780063
:105dd000214090000060a100a04098009e00780043
:105de000214090000000a1000010a1000020a100af
:105df000a04098009e007800314090000020a10053
:105e0000b04098001e007800be0090003108980055
:105e10001e0178006000b800000998001109980080
:105e20004e009000010020001e01780050019800f3
:105e3000610198009e0078000000eb00801098003f
:105e40001e0078009e009000210898001e00780037
:105e5000ae009000710098009e00780000c2b30070
:105e6000805898009e007800214090000070a100aa
:105e7000a04098000080fa00000006000a00fa0026
:105e8000000f780011079800220798003307980048
:105e9000440798009e007800214090000030a10047
:105ea000a04098009e007800214090000040a10092
:105eb000a04098009e007800214090000050a10072
:105ec000a04098009e007800214090000060a10052
:105ed000a04098009e007800214090000000a100a2
:105ee0000010a1000020a100a04098009e007800b2
:105ef000314090000020a100b04098001e007800c2
:105f0000be009000310898001e0178006000b800c3
:105f100000099800110998004e009000010020002f
:105f20001e01780050019800610198009e007800e1
:105f30000000eb00801098001e0078009e0090008a
:105f4000210898001e007800ae00900071009800b3
:105f50004e0090000000e00004003a009e0078002f
:105f600000c1b30080589800030037009e007800fd
:105f700000c3b300805898009e0078002140900034
:105f80000070a100a04098000080fa000000060008
:105f90000600fa00000f7800110798002207980009
:105fa0009e007800214090000050a100a040980081
:105fb0009e007800214090000060a100a040980061
:105fc0009e007800214090000000a1000010a10078
:105fd0000020a100a04098009e0078003140900071
:105fe0000020a100b04098001e0078009e009000a4
:105ff000310898001e0178006000b8000009980080
:10600000110998002e009000010020001e01780068
:1060100050019800610198009e0078000000eb009c
:10602000801098001e007800e008900000302000ea
:106030008080600000302000808f500004003a0013
:106040009e00780000c4b300805898000e0037000e
:106050001e007800e0089000003020008080600082
:1060600000102000808f500004003a009e0078004d
:1060700000c6b30080589800030037009e007800e7
:1060800000c8b300805898009e007800214090001e
:106090000070a100a04098000080fa0000000600f7
:1060a0000600fa00000f78001107980022079800f8
:1060b0009e007800214090000050a100a040980070
:1060c0009e007800214090000060a100a040980050
:1060d0009e007800214090000000a1000010a10067
:1060e0000020a100a04098009e0078003140900060
:1060f0000020a100b04098001e0078009e00900093
:10610000310898001e0178006000b800000998006e
:10611000110998002e009000010020001e01780057
:1061200050019800610198009e0078000000eb008b
:10613000801098001e007800e008900000302000d9
:106140008080600000302000808f500004003a0002
:106150009e00780000c5b300805898000e003700fc
:106160001e007800e0089000003020008080600071
:1061700000102000808f500004003a009e0078003c
:1061800000c7b30080589800030037009e007800d5
:1061900000c9b300805898009e007800214090000c
:1061a0000070a100a04098000080fa0000000600e6
:1061b0000e00fa0040479800310798004207980007
:1061c00053079800a048800010079800c14880003d
:1061d000010f78001ac8bf000044b2000004e000bc
:1061e0000f00320017c8bf000080fb004300dd0035
:1061f0008080e800a08d20000080400090017800a1
:106200005e009000010020000002be004e019000e0
:10621000be0090004e409000030001003e00370099
:106220003e00900060079800ee009000e18f500063
:10623000220032006e009000e10f40001f0032008b
:10624000330037001e009000500890000000e0006e
:10625000170032001e009000c05890004e009000c1
:106260006040900080cf500011003a001e00900066
:1062700050089000404090000080fb004300dd008b
:106280008080e800a08d2000008040009001780010
:106290005e009000010020000002be004e01900050
:1062a000be0090004e409000030001001a0037002d
:1062b0001e00900090007800110798001e009000ca
:1062c0000000e000dfff3a00130037001e007800f6
:1062d000404090000080fb004300dd008080e8002b
:1062e000a08d200000804000900178005e009000aa
:1062f000010020000002be004e019000be00900090
:106300004e409000030001001e007800100f78003e
:106310001e00e000edff3a000080fa0000000600d9
:106320001e00fa000000eb00300798008048800053
:10633000000f78000040eb00004f98000040eb0099
:10634000304f98001a28a9001a48a8001e007800ab
:1063500090407800415798001e0fe8001e0078001a
:1063600090407800615798001e0fe8001e007800ea
:10637000104078000080fb00600798001e0fe800c6
:106380001e007800104078000080fb004800dd000f
:10639000800078006e0090000100400060079800c7
:1063a0001e0fe8001e0078009040780021579800ea
:1063b0001e0fe8001e00780090407800214f9800e2
:1063c0001e0fe8001e0fe8001e0fe8001e007800f8
:1063d0009040780011579800790047009e50900037
:1063e00011409800f90047000040eb008048780019
:1063f000790147002400200005002000d100200082
:1064000000c0eb00191507000000e00005003a008d
:1064100080c2b30016e8b7000000eb00600f9800e0
:10642000450137004e5090008080fb003e009000f8
:106430000100400030079800814880003e00900035
:10644000008f40002a0137001e007800904078003d
:10645000415798001e0fe8001e0078009040780019
:10646000615798001e0fe8006e509000e94f5000f1
:106470000f003a001a28a8001e007800104078008b
:1064800013e8b70013c8bf000080fb000000d10074
:10649000610060000004e000050032001ac8bf007f
:1064a000684060000004e000010032001a48a900c2
:1064b0006e509000e44f5000090032004e509000a2
:1064c0008080fb003e0090000100400030079800f3
:1064d000814880003e009000008f4000040137009a
:1064e0001e00780090407800515798001e0fe80079
:1064f0001e00780090407800715798001e0fe80049
:106500001e00780090407800315798001e0fe80078
:106510001e00780090407800015798001e0fe80098
:106520001e00780090407800714f98001e0fe80020
:106530001e00780090407800614f98001e0fe80020
:106540001ac8bf000044b2000004e000030032009b
:1065500017c8bf00005f980014003700780047009c
:10656000800178006e499000fe4890000e50900027
:10657000fffa07000000e0000c003a003e489000df
:106580000040e800304f98004e5090008080fb00a3
:106590003e009000010040003007980081488000d4
:1065a0003e009000008f4000d10037008e489000e0
:1065b0005e50900080cf500004003a00be4890002a
:1065c0007e50900080cf5000090032004e50900065
:1065d0008080fb003e0090000100400030079800e2
:1065e000814880003e009000008f4000c0003700ce
:1065f00060002000d1f00700100798001e009000f6
:106600000000e00003003a000000eb00600f98007b
:10661000c90037001e009000de5090002140980015
:106620001e009000fe509000314098008e5890005f
:106630001e00900041409800c14880001e0090005c
:10664000010878001e009000c04888000e489000a5
:106650000040e800004f98000040eb00304f9800e9
:106660000040eb00104f98004e5090008080fb00df
:106670003e009000010040003007980081488000f3
:106680003e009000008f40008a0037001e00780016
:1066900090407800415798001e0fe8001e007800d7
:1066a00090407800615798001e0fe8006e509000ef
:1066b000e54f5000090032004e5090008080fb00f2
:1066c0003e009000010040003007980081488000a3
:1066d0003e009000008f400076003700200220002e
:1066e00096f00700200798002e0090000000e000c0
:1066f00003003a000000eb00600f98008e003700a6
:106700001e007800904078002e00900041589800bc
:106710001e0fe8001e007800904078002e009000c8
:10672000515898001e0fe8001e00780010407800b5
:106730008080fb002e009000410098001e0fe800b2
:106740002e009000c00090001e00780010407800dd
:106750000080fb004800dd00808040002e0090009b
:10676000410098001e0fe8001e00780010407800dd
:106770008080fb002e009000210098001e0fe80092
:10678000ae0090000000eb0090009800ae0090007a
:10679000314090000000a000b0409800ae00900092
:1067a000214090000070a000a04098002e019000b1
:1067b0006000b8000009980011099800ae00900030
:1067c0000040eb00805898002e0090009e00900042
:1067d000510898002e009000e00890000030200042
:1067e0008080600000102000808f50001b003a0065
:1067f0002e009000200090000000e00003003a000e
:10680000ae00900010002000a00098002e00900024
:1068100020009000f00f500003003600ae00900002
:1068200000012000a00098002e00900020009000a1
:106830000000e90080007800100020000100dd0069
:10684000800078002e00900021009800ae0090009b
:10685000314090000000a100b04098002e00900050
:10686000a00090002e00900031009800a048800009
:10687000900078002e00900001087800a048800069
:10688000ae009000010878001e4890000040e8002b
:10689000104f98004e5090008080fb003e0090000a
:1068a0000100400030079800814880003e009000c1
:1068b000008f4000be0090006e009000808f50005e
:1068c000040031009e4890003e50900080cf500060
:1068d0006eff39009e4890003e50900080cf5000df
:1068e000030032000000eb00600f98001200370038
:1068f000be0090006e009000808f5000d2fe3900e4
:106900008e4890002e50900080cf5000030032003f
:106910008000eb00610f9800070037002e489000c0
:1069200012e8b7001e5090000080fb00c0408800b5
:1069300011002000610f98006e0890000080fa009e
:10694000000006000400fa0020479800a0488000dc
:10695000000f78000e0037002e4090000004e00089
:10696000050032001e007800c05890002e409000b4
:1069700080cf500004003a009e0078003140900023
:106980000010a100b04098001e007800100f7800a1
:106990001e00e000f0ff3a000080fa000000060050
:1069a0000400fa002047980031479800d0c5b30092
:1069b000004f78001ac8bf00614060000004e0008a
:1069c0000200320000c8b3001e4f7000304080004b
:1069d00050589000634060000004e00002003a005c
:1069e000f0ceb3001e4f6000304080005058900041
:1069f00063406000e14f500002003a00e0cfb30076
:106a00001e4f60001e80fb005025880014c8bf0088
:106a10000080fb00b02488003e4090000080fb0016
:106a20004401dd002e4090008080fb00f007200034
:106a30000080600000007100f024880094a4a80089
:106a40000080fa00000006000600fa0040479800a7
:106a50004e409000e94f500017003a0000a020007f
:106a6000000f78001ac8bf00704060000004e0000a
:106a70000200320040a02000000f78001ac8bf00ba
:106a80000080fb004400de006140600000c0ea00be
:106a900061406000614060004401dd00a181200090
:106aa00091407800f0ceb30000c06000024070005a
:106ab0001ae8b7001600370080a02000000f780009
:106ac0001ac8bf000042b2000004e0000200320019
:106ad000c0a02000000f78001ac8bf000080fb0093
:106ae0004500de006140600000c0ea0061406000d7
:106af000614060004501dd00a181200091407800e7
:106b0000f0cdb30000c06000024070001ae8b7008a
:106b10004e409000ed4f50001a003a003040800087
:106b2000700090006101b800304080009008900033
:106b30000008900000015100818159003040800020
:106b40004000900001002000800f5100818f59000b
:106b50000400360030408000c0009000110798000b
:106b600023003700304080007001900030408000ea
:106b70009008900000089000000051001007980055
:106b80001b0037003040800050019000e001900071
:106b900030408000900890000008900000015100f3
:106ba00081815900304080004000900001002000a9
:106bb000800f5100818f5900040036003040800062
:106bc000c000900011079800090037003040800095
:106bd000e0009000500090000001780030408000fc
:106be00090089000000890000000510010079800e5
:106bf0004e409000ed4f500005003a0030408000bc
:106c0000a00890001e007800110098000a003700cc
:106c10003040800030089000000178003040800053
:106c2000900890000008900000004100800078006b
:106c30001e007800110098009e0078000040eb00d4
:106c4000904098009e009000f03f2000008160007e
:106c50009e01780013007800f13f200001016100df
:106c600001c02f0001006000020070008009780060
:106c700030408000304090000080fb000000d100d8
:106c8000614060009e017800930078000080fb0066
:106c9000610060004e01dd00f0ff2b00808060008d
:106ca0008280700081097800304080003040900080
:106cb000614060009e017800930078000080fb0036
:106cc000610060004b01dd00f07f2f0080806000dc
:106cd00082807000810978009e00780011007800a1
:106ce00000f0a000800878000080fa000000060094
:106cf0000400fa00a0488000000f78000b00370065
:106d00001e007800a040900000c8b30000c06000e2
:106d10000004e00003003a00100020001007980073
:106d2000060037001e007800100f78001e00e000fb
:106d3000f3ff3a000000eb00100798001e009000df
:106d40000080fa00000006003600f800809fbe00b8
:106d5000829fbe00849fbe00869fbe003400f80064
:106d600000c0b300a00188000a00fa00710480008e
:106d7000f0fb2f00008060007004880082c4bf0018
:106d80000044b2000004e0001000320080c4bf00e4
:106d90000044b2000004e0000c00320000042000b7
:106da00000248800204080000000e9002040880086
:106db000204080000000e00004003a0082c4a900e6
:106dc000e04080000000e800e04088008cc4bf0084
:106dd0000044b2000004e000100032008ac4bf008a
:106de0000044b2000004e0000c0032008cc4a90092
:106df0000004200050248800e140800000032000af
:106e0000808f500005003a00e140800000f0200033
:106e1000008060000010b000e04088008cc4bf001b
:106e2000614060000004e000090032008ac4bf0035
:106e3000614060000004e000050032001000200006
:106e4000502488008c04a9000000eb00f04088006a
:106e50008cc4bf00684060000004e0007201320092
:106e60008ac4bf00684060000004e0006e01320088
:106e70009024800030079800800020005024880073
:106e800030408000405890000080fb00ef00600020
:106e9000f02480006f006000808f500061013a0094
:106ea0003e009000680060000000e0000900320031
:106eb00080a02000100798003e0090006400600051
:106ec0000000e0000b003200c0a020001007980076
:106ed0000800370000a02000100798003e00900036
:106ee000640060000000e0000200320040a02000ca
:106ef000100798001e0090009000780000c023004a
:106f00008080600000802000808f500056003a0092
:106f10009e009000f03f20001100600020079800c4
:106f200034408000304080000009900090099000bb
:106f30002e009000010020000200400083804800e5
:106f4000000a9800110a9800314080000000eb0010
:106f50008010980030408000304090006240600017
:106f60000004e00005003200314080003140900014
:106f70000010a100b04098000400370031408000ac
:106f8000314090000010a000b040980030408000d8
:106f900000589000f04f50000a003200304080004e
